:0300000002006C8F
:10002300309822C0D075D008FFE9B42102743F1480
:10003300B50804C29C8009E599F608B83F02782107
:10004300C298EFD0D0309904D200C29932E509B5F5
:10005300080280FBF8E608B83F0278218809D29CA1
:10006300223000FDF599C20022E4F5D0F588F5A809
:10007300F59875813E758920758DFD858D8B438738
:1000830080D28E75984075A890D2007508217509A5
:1000930021D29C9000C47993E493A31164D9F911FC
:1000A30050B40312C2AF9000B1C082C0833290003B
:1000B30000C082C083321164B40DE4740A116480F9
:1000C300DE0D0A2A2A2A2A2053657269656C6C2080
:1000D3005472616E736D69742054657374206D6915
:1000E3007420313932303020426175643A0D0A0D83
:1000F3000A6162206E756E2077657264656E206199
:100103006C6C652065696E6765676562656E656EB3
:10011300205A65696368656E20616C732045636866
:100123006F207A757281636B676573636872696543
:1001330062656E2E0D0A4354524C2D43206681682E
:100143007274207A752065696E656D2052657365DA
:04015300743A0D0AE3
:00000001FF
